:100000001CC200000C94DF1B35C2000033C200008C
:1000100031C200002FC200002DC200002BC2000020
:1000200029C2000027C200000C94B7200C94832141
:100030000C94911A1FC200001DC200001BC20000D8
:1000400019C2000017C2000015C2000013C2000050
:1000500011C200000C94081B0DC200000BC200006E
:1000600009C2000007C2000005C2000003C2000070
:1000700001C20000FFC10000FDC10000FBC1000083
:10008000F9C10000F7C10000F5C10000F3C1000094
:10009000F1C10000EFC10000EDC10000EBC10000A4
:1000A000E9C10000E7C10000E5C100004A001E00F0
:1000B0001F00200021002200167C14001A000D00F1
:1000C0003600370050220C001800080012222D00C4
:1000D0004F213100380009000F2133430000000098
:1000E00034002E002A220400000000004C212B00C6
:1000F00091242C41230024002500260027004D00D8
:100100000A00070005001C001300E3001500173269
:10011000110016000B0052321D00103106001B00AA
:10012000190051310E0028322F003000000000006D
:100130002C4190344B004E31000000003A003B004F
:100140003C003D003E003F00010036002400250039
:1001500026000100010055002100220023000100BB
:10016000010035001E001F002000010000000000FB
:100170000100010001002700000000000100010053
:1001800001000100400041004200430044004500DE
:100190004B004A00CD004D00DD0001004E00CF00B5
:1001A000CE00D000DE000100D300500052004F000E
:1001B000DF000100D100D200510046000000000025
:1001C00001000100025201000000000029001E0091
:1001D0001F002000210022002B00170014001A002D
:1001E00008001500E1000A000400160007000900DD
:1001F000E000E2001D001B000600190000000000E6
:1002000010001C002C000B00000000001100180062
:1002100005000D0023002400250026002700000013
:100220000000000052000000E50000000000500047
:1002300051004F00E6000000000000000000000038
:10024000E40000004C002C00000000000000000052
:10025000280020520052D10000000000007C010064
:100260000100010001000100010001000100010086
:100270000100010001000100010001000100010076
:100280000100010001000100010001000000000068
:100290000100010001000100000000000100010058
:1002A0000100010001003A003B003C000100010098
:1002B00001003D003E003F00010001000100400040
:1002C00041004200010001000100430044004500DC
:1002D0000100010001000100010001000000000018
:1002E0000100010001000100000000002C03440097
:1002F00061006300740079006C002D004D00610006
:100300006E00750066006F0072006D00200028000E
:10031000350078003600290000000E0374007300D9
:1003200068006F00720074000000040309040902F1
:100330003B00020100A0FA090400000103010100D2
:100340000921110100012244000705810308000171
:10035000090401000103000000092111010001222C
:100360007B0007058203200001120100020000004B
:10037000084D44363501000102000105010902A1C2
:100380000185020901A100050919012908150025A7
:100390000195087501810205010930093115812592
:1003A0007F95027508810609381581257F950175AD
:1003B000088106050C0A38021581257F950175080C
:1003C0008106C0C005010980A101850319012AB772
:1003D00000150126B700950175108100C0050C09B4
:1003E00001A101850419012AA002150126A0029588
:1003F0000175108100C005010906A101050719E07A
:1004000029E71500250195087501810295017508F8
:1004100081010507190029FF150026FF00950675C3
:1004200008810005081901290515002501950575A4
:10043000019102950175039101C011241FBECFEFF8
:10044000DAE0DEBFCDBF11E0A0E0B1E0E2EAF8E41F
:1004500002C005900D92AA3AB107D9F722E0AAEAA4
:10046000B1E001C01D92A13DB207E1F70E943B132C
:100470000C94D723C5CD8430C8F46C30B8F4463022
:10048000A8F450E096E0699F400D511D112498E4B6
:10049000899F400D511D1124FA01EE0FFF1FE455F5
:1004A000FF4F85919491282F822F089521E090E0AD
:1004B000FBCFE1CF089581E0089581E00895FBCF5F
:1004C000089581E0089581E00895FDCF089508958D
:1004D0000895FDCF089508950895A6E0B0E0E3E7FC
:1004E000F2E00C944A2349835A839E833091B101F0
:1004F00089819A81311117C03E81311589F021150A
:1005000079F063D5182F682F89819A813DD569814B
:100510007A81812F0E94C60D2696E3E00C94662313
:1005200044D5182FF4CF51D569817A81F3CFFC01DE
:10053000262F408151816281738184819581CDCF45
:10054000CF93DF93EC0161E0F2DFBE01B6DF8115EE
:1005500029F061E0CE01EBDFBE01B1DFDF91CF9189
:1005600008950F931F93CF93DF93EC0160E0DFDFDB
:100570008C01BE01ADDFBE01C801ABDFDF91CF91C1
:100580001F910F9108950F931F93CF93DF93EC0169
:1005900061E0CDDF8C01BE0194DF811106C080E0F7
:1005A000DF91CF911F910F910895BE01C8018DDF9A
:1005B0008115A9F3BE01C8010E944118811579F384
:1005C000BE01C8010E94B814811549F3BE01C801DB
:1005D0000E948F14811519F3BE01C8010E940E0FED
:1005E0008115E9F2BE01C8010E94200F8115B9F200
:1005F000BE01C8010E943A0FD3CF21E030E002C013
:10060000220F331F8A95E2F7C901F9C3CF93C82F90
:1006100081E090E00C2E02C0880F991F0A94E2F747
:100620000E94E80B8C2FE9DFCF91089581E00895B7
:1006300081E00895FBCF0895CF93C82F8FD38C2FDF
:10064000F7DF8C2FF7DFCF91089581E0F5DF0C9471
:100650002C1B80E0F1DF0C943D1B3DDF0E94FA195A
:1006600017C018D039DF0C94FE1981E00895089561
:10067000CF93DF93C82FF9DFD82F811511F08C2F7E
:10068000F6DF8D2FDF91CF9108950895F1CF089572
:1006900080E0FCCF0E948818F9CFCF930E94881881
:1006A000C82F8091AC018C1771F0C093AC010E94EF
:1006B000FC1A6093AD017093AE018093AF019093EB
:1006C000B0018C2FE3DFCF910895ADE0B0E0EBE611
:1006D000F3E00C944B23488759876A877B878C8784
:1006E0009D8791118ED71F8286E0FE0138969E016C
:1006F0002F5F3F4FD90101900D928A95E1F78D81CF
:1007000081110CC029813A814B815C816D817E8190
:100710008F81C2D62D96E2E00C946723CE0101961C
:100720000FDF8111EFCFF6CFFC012481213019F4C6
:10073000808191817DC40895611521F00E94141675
:100740000C94C9160E945416FBCFCF93C82F811565
:10075000B9F08238B9F40E949D1881FD11C089E377
:100760000E945C19B7D78FEF97EE23E0815090403D
:100770002040E1F700C0000089E30E946219AAD777
:10078000CF910895833899F40E949D1880FDF8CF89
:1007900083E50E945C199ED78FEF91EE24E0815093
:1007A00090402040E1F700C0000083E5E6CF8438A8
:1007B00099F40E949D1882FDE3CF87E40E945C19A2
:1007C00089D78FEF91EE24E0815090402040E1F7EF
:1007D00000C0000087E4D1CF8450813A90F48C2F80
:1007E0000E94C3138111CCCF8C2F0E942019811538
:1007F00021F08C2F0E9462196DD78C2F0E945C19FA
:10080000BECF8C2F805E883048F481E0C1FD84E04B
:10081000C0FD880FC2FD8295D5D6B1CF8C2F855AE9
:10082000833030F48C2F8452990B0E94BE18A8CFCD
:10083000EC2FE85AEB3150F4F0E0EE0FFF1FE15DD2
:10084000FE4F808191810E94E5189ACF8C2F8D5C9C
:10085000833108F095CF61E08C2F6EDF91CF811549
:1008600009F44EC0823861F40E949D1881FF48C08F
:1008700089E30E945C192ED789E30E9462192AC776
:10088000833851F40E949D1880FF3AC083E50E948E
:100890005C1920D783E5F1CF843851F40E949D186C
:1008A00082FF2EC087E40E945C1914D787E4E5CF4D
:1008B000982F9450913A08F3982F905E983050F406
:1008C000982F81E091FD84E090FD880F92FD829544
:1008D0007FD6D5CF982F955A933020F480E090E0C2
:1008E0000C94BE18982F985A9B3120F480E090E029
:1008F0000C94E518982F9D5C933110F460E01CCFA8
:1009000008951F93CF93DF93182FEB011EDF2097DD
:1009100031F4812FA4DFDF91CF911F9108958FE9EA
:100920009FE00197F1F700C000002197F0CF60E54C
:1009300070E0893311F060E070E0E3CF811511F0D1
:1009400041D6C8C60895811511F042D6C3C6089590
:10095000A0E0B0E0EEEAF4E00C9445236C01D62F61
:10096000C72FFC011581068102950F7020D6E82E55
:100970008115E9F0E12E1115D1F08C2F807F8034A4
:1009800061F08D2F805E8830E0F08C2F807E803289
:1009900021F4D230B0F00115A1F08091A10282FFC4
:1009A00010C082E0B3D603D691E08927E82EEC2F61
:1009B000E295EF70C03C78F5F0E0E752FC4D0C9406
:1009C0003523E12CF4CF0C2F0F70C03110F00295BD
:1009D000007F111581F0011549F08D2F805E883060
:1009E00010F0D11105C0802FEDD574D68D2F40C0E9
:1009F000802FF9D5FACF8D2F32DF011561F08D2FC1
:100A0000805E883010F0D11103C0802FE1D502C084
:100A1000802FEFD55FD6E11409F4B3C0C4D580FDB3
:100A2000B0C0F6011582B9D51AD2C60168D1B5D5C4
:100A300024D2A7C08C2F8F70F82EC07FC03219F03F
:100A4000F29480EFF822D13038F079F1111509F4E1
:100A500038C00115C9F0CACF8091A10282FD10C033
:100A6000111541F0F11419F08F2DACD533D680E07B
:100A70006CDED1CF80E0F3DEF11469F28F2DC6CFAA
:100A8000111551F0013018F48F2D58DFC4CF09F043
:100A9000C2CF8F2DCAD5BFCF0111BDCF8F2D53DF50
:100AA0008F2DCED58F2DB3D5B6CF111521F00630B1
:100AB00008F0B1CFE9CF053008F0ADCF8F2D43DF7F
:100AC000AACF0115D9F3D93349F48FEF97EE23E07C
:100AD000815090402040E1F700C000008D2FBFDE24
:100AE0009ACF8C2F869586958370813060F009F0BF
:100AF00092CF8D2F9C2F9370111102C080E090E057
:100B00000E94E51888CF8D2F9C2F9370111102C081
:100B100080E090E00E94BE187ECF612F8D2F0CDE0A
:100B20007ACF8C2F8370C1F5111128C04D2F4295BB
:100B300046954770440F440F2D2F2F7030E0042E40
:100B400002C0220F331F0A94E2F780E090E0D4FF46
:100B500009C08FE090E002C0880F991F4A95E2F724
:100B600080959095C695C695C370822B932BC23005
:100B700079F0C33079F0C13049F04AD10E94881829
:100B800085DDCDB7DEB7E8E00C9461233AD1F6CF2E
:100B900046D1F4CF34D1F2CF111559F1C0FFEECFC9
:100BA0004D2F429546954770440F440F2D2F2F70BF
:100BB00030E0042E02C0220F331F0A94E2F780E0D7
:100BC00090E0D4FF09C08FE090E002C0880F991F29
:100BD0004A95E2F780959095C695C695C370822B8D
:100BE000932BC23061F0C33061F0C13031F06AD173
:100BF000C5CF823008F4C2CFD3CF5DD1BFCF69D18A
:100C0000BDCF1AD1BBCFCF70111529F08C2F27D1B2
:100C10008D2F94DEB3CF8D2F96DE8C2F2ED1AECFBD
:100C2000D23F31F168F4D03FC1F0D13F89F01115C6
:100C300009F43EC0011509F438C08D2F86DD9ECF22
:100C4000D33FE1F0D43F99F78091A10282FD1EC00D
:100C50008C2F8F71111511F30FC0111539F005305C
:100C600008F08CCF8C2F8F7118D188CF0630F8CF39
:100C70008C2F8F711111D2CFF2D080CF111521F0AE
:100C80008C2F8F71E3D07ACFDED078CF111529F079
:100C900063E08C2F8F7123D571CF81E037D502307F
:100CA00008F46CCF82E032D569CF8C2F8F71E4CFFE
:100CB000011571F0D93349F48FEF97EE23E081509D
:100CC00090402040E1F700C000008D2FC8DD56CFD6
:100CD0008C2F8F71A3CF0F931F93CF93DF93EC01D2
:100CE000688179818D81ADD18C01FAD087D0B8012E
:100CF000CE012EDEDF91CF911F910F910895CF93FA
:100D0000DF93EC018C81811581F0CE013CDC8111F7
:100D10000FC04DD4811549F08D81811531F080913E
:100D2000A10282FF02C082E0F1D4DF91CF91089549
:100D3000CE01D1DFCE0115DCF8CF80E090E00E943B
:100D4000BE1880E090E00E94E5185BD4C3D40E94F6
:100D5000E2160C94C9160E946819EFCF41D4FBCF5C
:100D6000282F92959F70963099F060F4925F9F7053
:100D7000923030F4203FB1F038F481E0283E38F072
:100D800080E008959A5FF3CF81E0243FC9F708958A
:100D900091E0813F09F090E081E0283E08F080E09A
:100DA000892B089581E00895FC012481211521F00B
:100DB000808191813DD1D4CF80E00895A6E0B0E05C
:100DC000E4EEF6E00C944B232696E2E00C946723C5
:100DD000A7E0B0E0EEEEF6E00C944B232796E2E0BD
:100DE0000C9467230895FECF0895FDCF0895FADF90
:100DF000FCDF8093D8019093D90108950895F7CF2F
:100E000008952091D8013091D901822B932BEFCFF7
:100E10002091D8013091D90182239323E8CF2091EA
:100E2000D8013091D90182279327E1CFDBCF0895F4
:100E3000FDCF0895D7CF0895FDDFFADF8093D60167
:100E40009093D701089580E090E0F6CF21E030E064
:100E500002C0220F331F8A95E2F7C901EDCF21E0CE
:100E600030E002C0220F331F8A95E2F78091D6014D
:100E70009091D701822B932BDFCF21E030E002C08D
:100E8000220F331F8A95E2F7209530958091D60185
:100E90009091D70182239323CFCF21E030E002C08D
:100EA000220F331F8A95E2F78091D6019091D701E6
:100EB00082279327C1CF2091D6013091D701822B71
:100EC000932BBACF2091D6013091D701822393235F
:100ED000B3CF2091D6013091D70182279327ACCF91
:100EE0000895CF93C1E061FDC4E060FDCC0F62FDC9
:100EF000C29593E0769567959A95E1F7660F771F0F
:100F0000660F771F460F571FFA0140E050E090E050
:100F10006191DF019C01042E02C0369527950A9449
:100F2000E2F72695220B26272C2326272E934F5FA8
:100F30005F4F4430510561F7CF910895A82FA770F6
:100F400023E0969587952A95E1F7880F991F880FDA
:100F5000991F680F791FFB0140E050E080E021916C
:100F600030E00A2E02C0369527950A94E2F72170E8
:100F7000042E01C0220F0A94EAF7822B4F5F5F4FC5
:100F80004430510561F70895262F9C3068F486306F
:100F900058F4682F70E086E0989F600D711D112451
:100FA00042EB51E0822F9DCF0895292F9C3058F4B9
:100FB000863048F490E062EB71E036E0239F800DCC
:100FC000911D1124BBCF80E00895CF92DF92FF9254
:100FD0000F931F93CF93DF936C010091D601109173
:100FE000D7018091D8019091D901082B192BCFE01E
:100FF000D0E081E090E00C2E02C0880F991F0A9487
:10100000E2F780239123892B61F4219790F7F12C4B
:101010008F2DDF91CF911F910F91FF90DF90CF9097
:101020000895FC2EB6018C2FBCD5019771F3F0CF3B
:10103000CF93DF93EC01C9DFBE01B3D5DF91CF9130
:1010400008950F931F93CF938B019091B101911548
:1010500031F0CB01EDDFCF911F910F9108958115F4
:1010600051F0CB01B2DFC82F682FC8018DDFB80166
:101070008C2F97D5F0CFCB0198DFC82FF8CF0F93E7
:101080001F930091DA018091DB01801303C01F914F
:101090000F91089587E0089FF0011124E452FE4F5C
:1010A000208131814281538164817581868190DE06
:1010B0000F5F1F4F0770E7CF209114023091150288
:1010C0004091160250911702609118027091190216
:1010D00080911A027DCE80911A02803170F4809145
:1010E0001902811551F0E091DA012091DB01309174
:1010F0001502409114022E1301C00895BF0187E02C
:10110000E89FF0011124DF01A452BE4F14968C9188
:101110001497811549F111968C911197831324C06E
:101120008C91841321C015968C91159781111CC048
:1011300012968D919D91A0911602B09117028A1B73
:101140009B0B883C910580F480911A028F7080611E
:1011500080931A02EE51FE4F80818F7080618083F0
:1011600084E192E0CCDD8BCF6F5F7F4FFB01E770B6
:10117000C2CF8F929F92AF92BF92DF92EF92FF9277
:101180000F931F93CF93DF93CDB7DEB72D970FB695
:10119000F894DEBF0FBECDBF8C0186E0F801DE0102
:1011A000189601900D928A95E1F7F801F5808481F7
:1011B00094E1892E92E0992E90911802911117C016
:1011C000811509F416C1F11409F455C1C801ECDD0B
:1011D000811509F450C187E0F801D40101900D9206
:1011E0008A95E1F7C401A0DA76DF66DF02C170817B
:1011F000A280B380D090190220911602309117027C
:10120000A501421B530BD11409F4F6C0483C51050B
:1012100008F0C5C0811509F4ECC030911502218198
:1012200080911A02803108F08CC0EF2C231326C065
:1012300030911402371322C0F11027C08F708061E3
:1012400080931A0239DF84E192E059DD80911A021D
:10125000F8018683E12C8E2D2D960FB6F894DEBF13
:101260000FBECDBFDF91CF911F910F91FF90EF90F7
:10127000DF90BF90AF909F908F9008958091DA019A
:101280003091DB01E82FF114D1F080911A028160D6
:1012900080931A02DFCFAF0167E06E9FF001112447
:1012A000E452FE4F6181261306C06081761303C0AD
:1012B00065816111EBC04F5F5F4FFA01E770E31387
:1012C000EACF381310C088859985B2DE292F229580
:1012D0002F709034E0F02A5F2F70223060F1C80147
:1012E0000EDDED2CB8CFAC0167E0869FF001112434
:1012F000E452FE4F8181281306C08081781303C019
:1013000085818111A7CF4395842F8770DACF9F7095
:10131000223038F0911551F0F8019681903130F477
:101320009ACF911519F0811509F495CF805E883018
:1013300008F491CFD4CF803F08F48DCF815F833004
:10134000F7CF231307C020911402271303C0F11411
:1013500009F473C0C80128DD811509F48CC0F114AB
:1013600009F489C080911A02803280F02091140221
:101370003091150229833A83AB82BC829091180286
:101380009D831E828F83CE010196B9DC87E0F80130
:10139000A4E1B2E001900D928A95E1F725CF20916A
:1013A0001A02203188F4488559856A857B858C85A9
:1013B0009D8504DD84E192E0A2DCF40187E01192D6
:1013C0008A95E9F779DE46CF811599F030911502BB
:1013D00081813813BFCF809114028713BBCFF110E6
:1013E000B9CF2683C8018BDCF40187E011928A957E
:1013F000E9F7EE24E3942FCF483C510508F03EC0B6
:101400008115B9F3F114B9F12091150281812813E6
:1014100029C080911402871325C080911A0280FD93
:1014200018C08031B0F08683807F803F39F086819C
:10143000982F907F905F8F70892B8683C8015FDC27
:1014400087E0F801A4E1B2E001900D928A95E1F7FE
:10145000CCCE87E0F801A4E1B2E001900D928A952C
:10146000E1F7C7CFC801A0DC811190CF80911A02AB
:10147000816080931A02C80142DCBBCF4885598540
:101480006A857B858C859D8599DC97CF84E192E088
:1014900036DCE4E1F2E092CFAEE0B0E0E2E5FAE083
:1014A0000C944A23288739874A875B876C877D8716
:1014B0008E87CE0108965DDE6C85811599F06115E9
:1014C00039F0288539854A855B857D858E8580DC68
:1014D0008091DA019091DB0189133DC02E96E3E003
:1014E0000C94662387E09E01285F3F4FF901275047
:1014F0003109D90101900D928A95E1F7611541F307
:10150000A091DB018A2F90E08395877090E0AC0179
:101510002091DA012417150691F097E09A9FD001E7
:101520001124A452BE4F9E012F5F3F4FF90101903D
:101530000D929A95E1F74093DB01A1DDC9CF0EDC56
:101540001092DB011092DA01E4E1F2E087E01192FF
:101550008A95E9F7BDCF17E0189FC0011124845286
:101560009E4F07DE811509F4B9CFE091DA011E9F85
:10157000F0011124E452FE4F2081318142815381D8
:1015800064817581868124DC8091DA019091DB0190
:10159000019687708093DA019BCF80912302869514
:1015A000869586950895809123028770089590917D
:1015B0002302977081E0911101C080E0089580912D
:1015C0002F02089590912F02982B90932F02089547
:1015D0008095982F80912F02892380932F02089560
:1015E00010922F02089590912E02982B90932E0224
:1015F00008958095982F80912E02892380932E0242
:10160000089510922E0208950895FECF08959091A6
:101610002402292F282329F08095892380932402EE
:10162000F4CF08950895FECF089590912502292FB3
:101630002823281721F0982B90932502F4CF0895A2
:1016400090912502292F282329F0809589238093C2
:101650002502E9CF089580912502811521F010928D
:10166000250280E0E0CF08950F931F93CF93DF937F
:1016700080910001909101018C01C0912F02809115
:101680002E02C82B80912502811529F0C82B0E94BB
:101690000C198111E0DFF801C083C0910001D091E5
:1016A000010148E050E06BE172E0CE010E94862328
:1016B000892B59F088E0FE01ABE1B2E001900D9278
:1016C0008A95E1F7CE010E949F18DF91CF911F917B
:1016D0000F910895C9CF08950895FECF0895909170
:1016E000A10292FF0EC0982F990F990F990F962B78
:1016F00090932302B4DB809123028695869586958C
:10170000ECCFADCB1092230280E0E7CF9091230283
:101710008095892380932302282F277059F48917F5
:1017200049F09091A10292FF05C086958695869515
:10173000A4DBE8CF08959091A10292FB222720F923
:10174000281749F080FB92F99093A10280EA92E079
:1017500043D082E0DBCF08958091A102002482FF74
:101760000394802DE8CF81E0E6CF80E0E4CF80E0F5
:1017700090E0BC01E6C380E090E0BC01DCD3F7CF91
:10178000A3E0B0E0E6ECFBE00C944B238DD398D3C0
:101790001B82CE010396ABD381E090E08093D80109
:1017A0001092D901B0D3198284E18A83CE010196C7
:1017B000BBD3E1DF2396E2E00C946723E1CF0895E9
:1017C00085C3089572C3089587C3089596C3089585
:1017D0009AC308959DC30895A7C30895B8C30895F3
:1017E000C0C30895A6E0B0E0E8EFFBE00C94492305
:1017F0000E94F01A8C018091300290913102801782
:10180000910779F019821A820E94F01ABC0149816D
:101810005A8180E090E00E946503009330021093AB
:1018200031022696E4E00C946523DAD26093360206
:10183000709337028093380290933902609332029A
:101840007093330280933402909335020895089583
:101850000895FDCF08950895FEDFFBCF0895FECFD4
:1018600008950895FEDFFBCF81E008958CE09FE0AE
:1018700012D7EEDFF1CF27C5089508950895089592
:10188000FCDFFCDFFCCF9EDF811101C097DF8AE324
:1018900092E09ADF80EA92E09DDF98DFB0DA8091F3
:1018A000D6019091D701C4CA0E94E71A70D20ED512
:1018B00053D4E9DF0E9486180E9445030E947514E4
:1018C00012D5D0CF00D581110C9487180895A6E0C9
:1018D000B0E0EDE6FCE00C944223C6DF81110AC0C3
:1018E00081DFF0DF0E9403170E944D032696EBE094
:1018F0000C945E234CD484E9A82E82E0B82E7501A6
:1019000010E0F7010081812F37D31F5F1C3009F4ED
:1019100045C09FEFE91AF90A081799F380913A0236
:1019200081FD30D3A8DF982E10E0812F25D3F82E2B
:10193000F50181915F01F81661F18F25D82E00E045
:10194000EE24E3948D2D8E21F1F0CC24C3948F2DC1
:101950008E2109F4C12C911489F0602F812F0E94EF
:101960004B1A81110BC009831A830E94F01ABC0123
:1019700049815A8181E09C2D0E9465034C2D602F86
:10198000812F0E945F1A0F5FEE0C0630D9F6F50129
:10199000F2921F5F1C3049F648DFA3CF0813BECF79
:1019A0009FCF0F931F93CF93DF93FDD0EC01D235E0
:1019B00008F050C0D03508F0C8C0C03ED10530F5A1
:1019C000CD3CD10508F09DC0C83AD10578F4C53AA0
:1019D000D10508F093C0C130D105B1F1CE01049713
:1019E000813A910588F1C0E0D0E02EC0CE01885A3E
:1019F00091094B97C0F7C85AD0E0CC0FDD1FCB59E7
:101A0000DE4F0990D881C02DD4641EC0D034A8F414
:101A1000D03208F0ADC0C83ED105B0F0CE01915033
:101A20009F3108F78D2F62D1082F8C2F90E0BBD00B
:101A3000D02FDF71C82FD92B07C08C2F90E0B3D0E7
:101A4000DF70C82FD92BD06ACE01DF91CF911F91C3
:101A50000F910895C03882E5D807B8F5C03682E501
:101A6000D80708F056C0C03482E5D807C8F4C032A1
:101A700082E5D80708F047C08C2F8695869520E22E
:101A8000829FC0011124C37021E030E002C0220F08
:101A9000331FCA95E2F7E901C82BD92BDD68D4CFF3
:101AA0008C2F86958695877020E2829FC001112435
:101AB000C37021E030E002C0220F331FCA95E2F765
:101AC000E901C82BD92BDC68BFCFC03C82E5D80721
:101AD00050F48C2F8F71C03AD24580F5982F84EF47
:101AE000906AEC01B1CFCE01805C9245809708F0FE
:101AF0007ACFDC2FDF71C0EFD06AA6CFA497D06475
:101B0000A3CFD065A1CF8C2F8F71D82FC1EFD06A12
:101B10009BCF8C2F86958695877020E2829FC0018F
:101B20001124C37021E030E002C0220F331FCA9598
:101B3000E2F7E901C82BD92BDA6886CFD7D0982FE6
:101B400080E09F71EC01D0627FCF8C2F8F71CED05F
:101B500053E0CC0FDD1F5A95E1F7DF70282F84FF8B
:101B600004C090E1899F90011124C22FD0696CCFED
:101B70008D2F8F71BBD0082F8C2F90E014D0302F79
:101B80003F71282F392B3062E9015ECF462F7C3020
:101B900028F4663018F4672F0C94590280E090E026
:101BA0000895F4DFFECE803E9105D1F1C8F4813373
:101BB000910509F481C048F48932910509F471C096
:101BC0008A32910509F47FC0089589339105E1F0C7
:101BD00082389105C9F08533910509F45DC00895F7
:101BE000843E9105D1F148F4823E910531F1833E66
:101BF000910541F181EE90E00895863E9105C1F195
:101C0000873E9105F1F108952091A002237009F01B
:101C100064C02091A10223FF14C089E290E00895DE
:101C20002091A00220FD45C03091A10230FF09C0E3
:101C300024FD24C083EE90E008952091A00222FDAF
:101C4000F7CF08952091A00222FD44C03091A10257
:101C500030FD43C024FFF5CF11C02091A10221FF28
:101C6000F0CF8091A00284FD09C087EE90E0089536
:101C70002091A00223FFE5CF24FFF7CF80E090E082
:101C800008952091A00223FD2BC03091A10231FFC5
:101C9000E1CF84EE90E008952091A00225FFD1CFFE
:101CA000BCCF2091A00225FD1EC02091A10223FFE0
:101CB000C8CF89E390E008952091A00226FFC1CF0C
:101CC0008AE290E008952091A00226FFBACF81E336
:101CD00090E0089582EE90E0089580EE90E00895FF
:101CE00086EE90E0089585E390E008959091A0023B
:101CF00092FF10C041E0282F2471243009F040E009
:101D000031E0282F2871283009F030E0431711F016
:101D10002CE0822793FF10C041E0282F247124314A
:101D200009F040E031E0282F2871283109F030E037
:101D3000431711F02CE082273091A10230FF10C030
:101D400051E0282F2171213009F050E041E0282F87
:101D50002871283009F040E0541711F029E082275B
:101D600031FF10C041E0282F2171213109F040E0FE
:101D700031E0282F2871283109F030E0431711F0A5
:101D800029E0822794FF02C083FD877E0895109288
:101D9000A2021092A3021092A4021092A50208952A
:101DA000EF92FF920F931F937B018C018CD28111D4
:101DB00012C00E94FC1A9701A801261B370B480B82
:101DC000590BC901DA018093A2029093A302A09358
:101DD000A402B093A5021F910F91FF90EF90089578
:101DE00072D2811541F00E94FC1A462F572FBC0178
:101DF000CB01BA0108950E94FC1ADC01CB0140918D
:101E0000A2025091A3026091A4027091A502480F12
:101E1000591F6A1F7B1FECCF80E00895CF939C0170
:101E2000205E3245C1E02032310538F4FB01C58126
:101E3000C11103C08F710E9406038C2FCF910895AA
:101E40009C01FB018581811599F02B359CE73907B1
:101E500069F02C359CE7390721F02A353C4721F001
:101E600008957ADC80E008957EDCFCCF7EDCFACF3A
:101E700081E008959C01FB018581811599F0213055
:101E80009CE7390761F023309CE7390739F02115C9
:101E90003C4749F40E94250380E0089591DC0E94AC
:101EA0002903FACF81E00895089580E090E00E9430
:101EB000A4239C0181E0233E3E4F09F080E0089579
:101EC00063EE7EEF80E090E00C94C3236FEF7FEF32
:101ED00080E090E00C94C323CF93DF93EC0182E089
:101EE00090E00E949C238883DF91CF910895FC01AC
:101EF000608182E090E00C94A92383E090E00E944E
:101F00009C2390E00895682F83E090E00C94A9232F
:101F1000CF93DF93EC0184E090E00E94A4238883B8
:101F20009983DF91CF910895FC016081718184E0F4
:101F300090E00C94C323AB01BC018FE090E00C94C3
:101F4000BB23AB01BC0183E190E00C94BB238EE08A
:101F500090E00E949C23982F81E0911101C080E0C5
:101F60000895682F8EE090E00C94A9230895FECF89
:101F700008950895FECF0895E82FF0E0ED54FD4F49
:101F800080810895089580EA8A95F1F7089500C048
:101F90000895F9CF08950895FECF0895A6E0B0E022
:101FA000E4EDFFE00C9446238ED1F82E8091BF0221
:101FB00090E08D549D4FF114E1F18E010F5F1F4FA2
:101FC000F80126E011922A95E9F7B80198D1E02EA0
:101FD000D12E8115B1F08091A60290E046E050E04C
:101FE000B8018D549D4F0E94862321E020933B022F
:101FF000892B91F4F12CBEDF8F2D2696E7E00C940F
:10200000622380913B028115A9F3F80186E01192C9
:102010008A95E9F710923B02A091A602B0E0AD5478
:10202000BD4F86E0EE2DFD2D01900D928A95E1F7D2
:10203000E2CF2091A60230E0BC01C9018D549D4F32
:10204000E9D1AADFD9CFF894E82FE295EF70F0E05C
:1020500041A18F7021E001C0220F8A95EAF7922FEB
:102060009095942391A392A1822F892B82A3789497
:102070000895CF93DF93C1EAD1E089918F3F09F0B2
:10208000E2DF81E0C73AD807C1F7CBE9D1E0899117
:102090008F3F09F0D8DF81E0C13AD807C1F7DF915F
:1020A000CF910895A0E0B0E0E8E5F0E10C9445237D
:1020B0006C01E62EC62FD0E08E010F551E4FF801A1
:1020C00080818F3F09F441C0F894E82FE295EF70CA
:1020D000F0E091A18F7021E001C0220F8A95EAF70C
:1020E000892F822B81A382A12095282322A3789473
:1020F0004EDFABE9B1E031E0F12C2D912F3F79F0CB
:10210000E22FE295EF70E05EF0E0808190E02F70CA
:1021100002C0959587952A95E2F780FF1BC080E065
:10212000F82A330F81E0A13AB80739F7F801808126
:102130008F3F09F088DF61E0F11001C060E08E2D73
:1021400028DFF601EC0FFD1FF082CDB7DEB7E8E027
:102150000C946123832FE4CFB3D0B2D090E08111EF
:1021600001C096E09093BF0286E0891B8093A6028F
:1021700080DFE3EBF2E08CE011928A95E9F7E7EA81
:10218000F2E08CE011928A95E9F741D0F0CEACE014
:10219000B0E0EDECF0E10C944823FE013196DF0154
:1021A0008CE01D928A95E9F710E00E2FFF2E612F2B
:1021B000802F9F2D77DF812F8F5F182F8630B9F703
:1021C0004CE050E0602F7F2D87EA92E00E9486234A
:1021D00041E0892B91F440E06091BF0270E06D54C2
:1021E0007D4F87EA92E014D0182FD8DE912F982BDC
:1021F000892F2C96E5E00C9464238CE0E02FFF2DD2
:10220000A7EAB2E001900D928A95E1F7E5CF089533
:10221000EF92FF920F931F93CF93DF938C017B017B
:10222000C42F411579F081E080933E020E94F01A9C
:1022300080933C0290933D0280E0CDB7DEB7E6E0AC
:102240000C946323D0913E02D115B1F380913C02EE
:1022500090913D020E946F1A059770F346E050E09E
:10226000B801C7010E948623892B41F086E0F8015E
:10227000D70101900D928A95E1F7CD2F10923E0281
:102280008C2FDBCF9FDA811101C098DAA7CA1F9388
:10229000CF93DF93C8ECD0E00E941C23182F81114C
:1022A0000AC08FE39CE90197F1F700C00000219775
:1022B00099F70E941823812FDF91CF911F910895E4
:1022C000809142020895809141020895E0DF809359
:1022D0004102D8DF80934202F3DF80930201F3DFF3
:1022E000811140C00895EFDF811101C03EC0089503
:1022F00081E0909143029A3008F080E008950F93B6
:102300001F93CF93DF93EC018B01809143028A30BE
:1023100080F4B801CE017CD0811121C080914302AC
:102320008F3FB1F40E94F01A80933F0290934002D5
:1023300009C080913F02909140020E946F1A843F31
:10234000914038F780E0DF91CF911F910F91089570
:102350008F5F809343028A3028F781E0F4CF109298
:102360004302FBCF0C949B1B08950C949E1B089575
:10237000CF92DF92FF920F931F93CF93DF93690168
:10238000E801082F880F110B41155105B1F0F80134
:1023900033E0EE0FFF1F3A95E1F7ED5FFE4F8181CD
:1023A00092818C5B9D4FE0812E2F30E04E175105BE
:1023B00008F49A01A9010E949323C8010E947C1C81
:1023C000F82E8115E1F02097D1F0C80123E0880FA5
:1023D000991F2A95E1F7FC01ED5FFE4F2381422F03
:1023E00050E0C217D10508F4AE018D5F9E4FFC018D
:1023F000648175816C5B7D4FC6010E9493238F2D94
:10240000DF91CF911F910F91FF90DF90CF900895B2
:10241000E9C00895FCC00895A4E0B0E0E2E1F2E173
:102420000C94492360915D0270915E0280915F027D
:10243000909160020E94781A11E06436710581055E
:10244000910508F1CDDCDC01CB010296A11DB11D87
:1024500089839A83AB83BC8300E010E0980144E059
:1024600050E0CE010196BC0182E082DF182F811579
:1024700051F00E94FC1A60935D0270935E0280939B
:102480005F0290936002812F2496E4E00C94652310
:10249000A7E0B0E0EEE4F2E10C9443235B01E090AE
:1024A000A701F090A80101E010E0CE0107969C0181
:1024B00040E050E0BA0180E05BDF182F811509F49D
:1024C00045C067018FEFC81AD80A60915902709110
:1024D0005A0280915B0290915C020E94781A6436E5
:1024E00071058105910558F106E010E0CE010196D5
:1024F0009C0140E050E0BA0181E03ADF182F66E02D
:1025000070E0C601F3D19F8198132DC0111559F1C8
:102510000E94FC1A6093590270935A0280935B02E6
:1025200090935C0286E09E012F5F3F4FF901A3E587
:10253000B2E001900D928A95E1F781E015C066E066
:1025400070E0C601D3D19F818913CECF86E0F70119
:1025500031969E012F5F3F4FD90101900D928A95D0
:10256000E1F71111DFCF80E096E0E3E5F2E0D5017D
:1025700001900D929A95E1F72796EAE00C945F237B
:10258000A0E0B0E0E6ECF2E10C9443237C016B01A7
:102590005A01AEDE0AE010E0811102C001E010E055
:1025A000C1E0D0E0B601C701F5010995811115C060
:1025B00021960C171D078CF0CC9F9001CD9F300DFC
:1025C000300D112480E090E045E34A95F1F70000DA
:1025D000019682179307C1F7E5CFCDB7DEB7EAE0E2
:1025E0000C945F230F931F93CF93DF93EC018B0128
:1025F00048E452E1C5DF811529F04CE052E1B80111
:10260000CE01BEDFDF91CF911F910F910895CF933F
:10261000DF93C091A701D091A801CE01019626E0D9
:10262000FB01DC0101900D922A95E1F766E070E074
:102630005DD188838F819885A985BA8540914F02A5
:102640005091500260915102709152028417950787
:10265000A607B70759F080934F0290935002A093BA
:102660005102B0935202BC01CD019ADBDF91CF91B0
:1026700008952DC908954ED70E940C1EF7D80E94C8
:10268000241E12D90E942D1E0E94301EF2DF0E94CD
:10269000501EF6D8F9CF8093AA019093AB0108950C
:1026A0008B3258F4853098F0E82FE550E63278F414
:1026B000F0E0EB51FC4D0C943523833450F48A3315
:1026C00008F051C0853331F091E0883361F090E03B
:1026D0000AC0E9F781E090E00E94FF060E94AE0682
:1026E00001C06CD891E0892F089580913A02807FD3
:1026F00080933A0281E080936402F4CF0E94250324
:10270000F1CF90913A02892F8E7F90FF8160809364
:102710003A0280FDE7CF817F80933A02E3CF909128
:102720003A02892F8D7F91FF826080933A0281FF68
:10273000D9CF80913A028160EFCF90913A02892FF0
:102740008B7F92FF846080933A0282FDF2CFCACFE2
:1027500090913A02892F877F93FF886080933A0295
:1027600083FDE7CFBFCF895321E030E002C0220FC5
:10277000331F8A95E2F7C901AFCF8D51F5CF80E0C5
:10278000089580E00895CF93C82F8091640281302E
:1027900089F0823081F18111A4C00E94DF0A823267
:1027A00009F0A1C08C2FEBDF811102C08C2F78DFE4
:1027B000CF9108950E94DF0A8232A1F38C2FE1DFCE
:1027C000811519F081E08170F3CFC43169F030F4E4
:1027D000CB30C1F3C03159F080E0F5CFC93221F0E0
:1027E00081E0C833C9F7EFCF10926402F5CF82E0E1
:1027F00080936402E7CFCF3409F469C068F4C8322B
:1028000048F4CE3178F5C73009F450C0C431F9F03E
:1028100081E0CECFC932FBCFC13509F45AC0C235F1
:1028200009F459C086EFC03599F7E0916102F09143
:102830006202309769F32081982F990F990B820FCC
:10284000911D91300CF449C08FEF8083E1CF8091CE
:1028500063028115E9F210926302109261021092F4
:102860006202D6CFCD51C0936302C430C9F078F470
:1028700080E291E0C23031F087E692E0C33011F49B
:102880008FE191E08093610290936202C1CFC530E5
:1028900051F08BE191E0C630A9F310926302B8CFFA
:1028A0008EE191E0EFCF8CE191E0ECCF10926702E6
:1028B00084E180932001C0931F018CE380931E016B
:1028C00088E080931C0188E280931B01A1CF8AE0FD
:1028D000ACCF8FEFAACF81E0A8CF97FFB6CF108201
:1028E00097CF1092640280E063CF0895FC01680FD7
:1028F000791F8FEF41E3E617F70709F408959191E7
:10290000892728E030E0982F990F87FF06C0892F8C
:10291000842721503040B9F7EECF892FFACFCF93DB
:10292000DF93EB0186319C4709F50E94DF0A9D8108
:10293000911599F08A7A91E0811101C090E090930D
:102940006502811541F085E3B7D40E946A0B80E0EF
:10295000DF91CF91089589E2F7CF809165028115CB
:1029600019F085E3AFD4F1CF89E2FCCF81E0F0CF5D
:10297000CF93DF93EC01FB018581811509F4CBC076
:102980009E0130572332310508F0ABC080EA92E057
:102990000E94EA0BFE01E150F047E232F10520F41B
:1029A000E55FFB4D0C9435238091A00281608093FC
:1029B000A00290C08091A10288608093A1028AC089
:1029C0008091A0028260F3CF8091A0028460EFCF5B
:1029D0008091A0028860EBCF8091A1028160EDCF51
:1029E0008091A1028260E9CF8091A0028061DFCF57
:1029F0008091A0028062DBCF8091A0028064D7CF5B
:102A00000E94AE068091A0028068D1CF8091A00282
:102A10008C60CDCF8091A1028360CFCF8091A00246
:102A20008E7FC5CF8091A102877FC7CF8091A00202
:102A30008D7FBDCF8091A0028B7FB9CF8091A00206
:102A4000877FB5CF8091A1028E7FB7CF8091A10201
:102A50008D7FB3CF8091A0028F7EA9CF8091A002FD
:102A60008F7DA5CF8091A0028F7BA1CF0E94AE0663
:102A70008091A0028F779BCF8091A002837F97CF18
:102A80008091A1028C7F99CF9091A002892F8B7F9A
:102A900092FF8460877F92FF886089CF8091A10236
:102AA000982F909590FB80F990FB81F986CF9091BB
:102AB000A002892F8F7B96FF806479CF0E94AE069B
:102AC0009091A002892F97FB87F9805870CF81E001
:102AD0000E94F00B80EA92E00E94EC0B0E94AE068E
:102AE00080E0DF91CF91089580E0F2CF9091A00235
:102AF000892F8F7E94FF80615ACF9091A002892FF9
:102B00008E7F90FF816053CF9091A102892F877FA4
:102B100093FF886052CF81E0E4CF382F25EB32035A
:102B2000C001112497FF04C080589109892F08958E
:102B300080589F4FFBCF80916E0280FF0DC0609147
:102B40001F0170E0660F771F6038710588F5611509
:102B5000710581F1862F089581FF07C060911F01E3
:102B600084E0689FB0011124EFCF82FF04C0609120
:102B70001F0188E0F6CF90916D029115B9F0609138
:102B80001E0180911F01961728F098E0899FB001DF
:102B90001124DACF899FC001112423E0880F991FE7
:102BA0002A95E1F770E00E942223CECF68E0D2CFD1
:102BB0008FE7089581E0089580916E0280FF0CC038
:102BC00060911C0170E07595679575956795611525
:102BD000710541F1862F089581FF06C060911C01A7
:102BE00070E075956795F3CF60911C0182FD0BC075
:102BF00090916C029115A1F060911B0180911C01D4
:102C0000961738F0682F70E06038710500F38FE791
:102C10000895899FC001112470E00E942223F4CFFF
:102C200061E0D8CF81E00895E82FED5CE33198F5BD
:102C3000F0E0E35DFB4D0C9435237DDF81958093BF
:102C40007202089578DFFBCF76DF81958093710261
:102C5000089571DFFBCFB0DF809373020895ACDF7E
:102C60008195FACFA9DF8195809374020895A4DF3E
:102C7000FBCF815D990B21E001C0220F8A95EAF715
:102C800080917002822B80937002089580916E0271
:102C9000816080936E02089580916E028260F9CF08
:102CA00080916E028460F5CF409171028D3C59F4A1
:102CB0008091720287FF0DC010927202411559F483
:102CC00010926D0208C08E3C81F480917202181639
:102CD0009CF3411581F08091730290917402892BCD
:102CE00009F056C010926C0208958F3C41F447FFE2
:102CF000F0CF10927102809172028115E0CF803D79
:102D000019F41416B4F3E5CF90917302893D29F4B8
:102D10001916FCF610927302DCCF8A3D19F497FF66
:102D2000D8CFF8CF909174028B3D29F497FFD1CF83
:102D300010927402CECF8C3D19F41916CCF3C9CF82
:102D4000982F915D983078F4815D990B21E001C056
:102D5000220F8A95EAF7822F80959091700289233D
:102D600080937002B6CF8D3D31F480916E028E7FDC
:102D700080936E02AECF8E3D21F480916E028D7FE6
:102D8000F7CF8F3D09F0A5CF80916E028B7FF0CFFA
:102D9000089526D49C019091710280917202982B23
:102DA00021F020936A0230936B029091730280911C
:102DB0007402982B21F020936802309369028FE609
:102DC00092E0CAC1EFE6F2E086E011928A95E9F757
:102DD00010926D0210926C0210926E020895FC0126
:102DE000828181110EC0838181110BC08481811188
:102DF00008C091E08581811101C090E0892F817028
:102E0000089581E0FCCFA6E0B0E0E9E0F7E10C94A2
:102E1000482386E0EFE6F2E09E012F5F3F4FD901A5
:102E200001900D928A95E1F7109271021092720250
:102E300010927302109274028B819C81892B022F55
:102E4000F32E811581F080916A0290916B0247D335
:102E5000AC0190916D029115A1F180912001841730
:102E6000150608F43BC08D819E81892B89F08091E5
:102E700068029091690233D3AC0190916C02911574
:102E800009F45AC080911D018417150608F462C028
:102E9000602F7F2D8FE692E025D2811104C08FE64E
:102EA00092E09DDF811175DF86E0E02FFF2DAFE618
:102EB000B2E001900D928A95E1F72696E5E00C9438
:102EC0006423209167028AE0289F9001112424172F
:102ED000350748F69F5F90936D0202C09F3FD1F780
:102EE0001B81111551F027DE91E011160CF09FEFB8
:102EF000899F802D1124809371021C81111551F03E
:102F00001ADE91E011160CF09FEF899F802D11249D
:102F10008093720280917102811509F4A4CF1091FF
:102F20007202111509F49FCFF8DD80937102812F91
:102F3000F4DD8093720297CF209166028AE0289F89
:102F4000900111242417350708F0A2CF9F5F9093BA
:102F50006C0202C09F3FD1F71D81111551F02CDE8C
:102F600091E011160CF09FEF899F802D1124809322
:102F700073028E81182F811551F01EDE91E011161B
:102F80000CF09FEF899F802D112480937402809113
:102F90007302811509F47CCF90917402192F911559
:102FA00009F476CFBADD80937302812FB6DD80936A
:102FB00074026ECF0F931F93CF93DF93C42FD22F42
:102FC000FC0185818115C9F04093770209D3809374
:102FD0007502909376028C2F805E883048F481E0F1
:102FE000C1FD84E0C0FD880FC2FD82950E949E0451
:102FF000DF91CF911F910F910895109177021413D3
:1030000033C0809175029091760269D2883C910517
:1030100058F5CD2FC05E1D17C1F0812F805E88301E
:1030200048F481E011FD84E010FD880F12FD8295C7
:103030000E94A304C83048F481E0D1FD84E0D0FDB3
:10304000880FD2FD82950E949E04802F0E949704D3
:1030500081E0D1FD84E0D0FD880FD2FD8295C8309B
:1030600038F60E94A304C4CF8C2F805E883008F00D
:10307000BFCF81E0C1FD84E0C0FD880FC2FD829515
:10308000F0CF0F93FC01CB01E851FC47E730F1058D
:1030900088F5E05CFB4D0C94352306E221EE41EE11
:1030A0006AE17CE787DF80E00F91089507E225EE73
:1030B00045EE6BE17CE7F6CF06E221EE40EE68E1FB
:1030C0007CE7F0CF07E225EE44EE69E17CE7EACF4A
:1030D00006E221EE42EE6CE17CE7E4CF07E225EE6A
:1030E00046EE6DE17CE7DECF08E221E045EE6EE1E1
:1030F0007CE7D8CFFB01858181111092770281E0B6
:10310000D3CF80937D0290937E0208950895089511
:10311000DAD8811103C0809178020895E0917D0290
:10312000F0917E02309739F00190F081E02D3097D8
:1031300011F00995089580E00895EACF0895E0918F
:103140007D02F0917E02309731F00280F381E02D14
:10315000309709F009950895E0917D02F0917E0283
:10316000309759F026813781232B39F022E0DC019A
:103170002C930680F781E02D09950895A3E0B0E037
:10318000E4ECF8E10C944B2320917B0230917C021B
:1031900028173907B1F080937B0290937C02E0916D
:1031A0007D02F0917E02309761F00084F185E02D80
:1031B000309739F023E029838A839B83CE010196DF
:1031C00009952396E2E00C946723A3E0B0E0EBEED0
:1031D000F8E10C944B232091790230917A02281760
:1031E0003907B1F08093790290937A02E0917D02E1
:1031F000F0917E02309761F00084F185E02D3097E8
:1032000039F024E029838A839B83CE0101960995B6
:103210002396E2E00C946723409100015091010154
:103220009A012E5F3F4F485F5F4F80E0F901908128
:103230002F5F3F4F91118F5F42175307B9F70895E2
:10324000811591F02091000130910101F901329630
:10325000285F3F4F9081981731F03196E217F307BE
:10326000C9F780E0089581E008959C01FC01329641
:1032700080E09FEF4081461759F031969F3F19F447
:10328000411101C0982F8F5F8630A1F79F3F09F44D
:103290000895290F311D97FD3A95F901628308952C
:1032A000FC01329608962191261302C0DF011E927E
:1032B000E817F907C1F70895682F809100019091F0
:1032C0000101D3CF682F8091000190910101E8CFD7
:1032D000E0910001F0910101329686E011928A9509
:1032E000E9F70895DC01FB0111969C91119781810A
:1032F000981322C012968C911297811519F0928121
:1033000089131AC013968C911397811519F0938124
:10331000891312C015968C911597811519F0958116
:1033200089130AC014969C91911521F081E02481A3
:10333000291303C080E001C081E0817008950895E1
:10334000FECF08958F5F80932401609121017091D9
:1033500022018091230190912401F2CF83E0809398
:1033600024016091210170912201809123019091AB
:103370002401E6CFE7CF089581E080932401609196
:103380002101709122018091230190912401D8CFD5
:10339000F3CF089591E0811101C090E09093230153
:1033A000609121017091220180912301909124016B
:1033B000C7CF80912301089580932201609121015C
:1033C000709122018091230190912401B9CF8091C5
:1033D00022010895809321016091210170912201C1
:1033E0008091230190912401ABCF80912101089518
:1033F00008950895FECF089508950895F9CF08958A
:103400000F931F93CF93DF93F7DF0E94C710F5DF71
:103410000FE712E0C0E0D0E08C2F0E94BC0FF80153
:1034200081938F0191E0811101C090E0D92BCF5F92
:10343000CC3091F78D2FDF91CF911F910F9108958F
:10344000EF92FF920F931F93CF93D6DF0E94C71086
:10345000D4DF8FE7E82E82E0F82E04E912E0C0E026
:103460008C2F0E94BC0FF70131917F01F80121914F
:103470008F01F701922F90959823932B9293F80147
:10348000282B2293CF5FCC3059F7CF911F910F910A
:10349000FF90EF900895E82FF0E0E158FD4F808114
:1034A00090E021E030E002C0220F331F6A95E2F77E
:1034B0002823392381E0232B09F480E0089541116A
:1034C0000DC0E82FF0E0E158FD4F21E001C0220FD0
:1034D0006A95EAF720958081282320830895CF9369
:1034E000DF93EC017DD08C1B9D0BDF91CF91089574
:1034F000EF92FF920F931F937B018C017DD0970178
:10350000A801621B730B840B950B1F910F91FF9009
:10351000EF90089585B7806885BF85B7806885BFBF
:1035200008951F921FB61F9211248F939F93AF93FC
:10353000BF9380918B02811113C08091C002909142
:10354000C102A091C202B091C3024196A11DB11D5A
:103550008093C0029093C102A093C202B093C302B1
:10356000BF91AF919F918F911F901FBE1F90189593
:103570008091C802843031F10E942D0310928B0299
:1035800088E190E020E40FB6F894A895809360005D
:103590000FBE2093600083B7817F846083BF83B7B1
:1035A000816083BF7894889583B78E7F83BF0FB681
:1035B000F894A895809160008861809360001092D3
:1035C00060000FBE08950E94AE060C94310382E0A5
:1035D00084BD93E095BD9AEF97BD80936E000895EA
:1035E0002FB7F8948091C0029091C102A091C202BD
:1035F000B091C3022FBF08952FB7F8946091C00215
:103600007091C1028091C2029091C3022FBF0895B0
:1036100078941F921FB61F9211248F939F93AF939C
:10362000BF938091C0029091C102A091C202B0915B
:10363000C3020196A11DB11D8093C0029093C102E7
:10364000A093C202B093C302BF91AF919F918F919B
:103650001F901FBE1F90189587E797E7809300087B
:103660009093010888E19AE00FB6F894A8958093AA
:1036700060000FBE90936000FFCF88E19AE00FB624
:10368000F894A895809360000FBE90936000FFCFE0
:103690008EE1489B02C08150E1F7489BFECF089520
:1036A000589880E28A95F1F7589A0895FC018BE0CA
:1036B0008A95F1F798E020E080E031E040E14A951A
:1036C000F1F7880F489B02C08160232742E04A95AA
:1036D000F1F7000040E14A95F1F7915079F790E158
:1036E0009A95F1F799B132E03A95F1F7000030E19F
:1036F0003A95F1F7917092272081920F9083089567
:10370000A1E0B0E0E5E8FBE1C2C719828C017C01D1
:10371000E60EF11CBDDFCE010196C8DFF8018193F2
:103720008F01EE15FF05B1F781E09981911180E0DD
:103730002196E6E0C8C7509A589A08955098589A2A
:10374000E89AE9E6F0E080818C7F808308956150FB
:10375000770B91E001C0990F6A95EAF7692F90E025
:1037600021E0611108C0911591F0589A80E28A9584
:10377000F1F758980895362F382339F0589A922740
:1037800030E23A95F1F76695ECCF5898F9CF589812
:10379000EDCFFF920F931F93CF93DF93EC018C013A
:1037A000060F111D8991F82E7BDF68E08F2DCFDF8A
:1037B000C017D107B9F7CDB7DEB7E5E085C71F92CF
:1037C0000F920FB60F9211240F931F932F933F93D5
:1037D0004F935F936F937F938F939F93AF93BF9319
:1037E000EF93FF93CF93DF930F92CDB7DEB719829C
:1037F0004FDFCE0101965ADF082F069506950695F4
:10380000282F22952570902F9570920F292F2370C5
:1038100096959695920F982797708981892B09F034
:1038200055C0043008F052C080E18A95F1F7589AEB
:10383000509A82E08A95F1F700C0589888E0089F76
:1038400080011124D801AD5FBE4F1696ED91FD9118
:103850001897309791F06091A7017091A801149684
:103860002D913D91260F371F15978D919D91680FD2
:10387000791F4C9113978C910995F801ED5FFE4FDC
:103880006381611549F02091A7013091A8018481DD
:103890009581820F931F7DDF03DF80E18A95F1F729
:1038A00058985098589A80E18A95F1F7F801ED5FA1
:1038B000FE4F6081611549F02091A7013091A80168
:1038C00081819281820F931F1BDFE2DE0F90DF91D7
:1038D000CF91FF91EF91BF91AF919F918F917F9188
:1038E0006F915F914F913F912F911F910F910F9089
:1038F0000FBE0F901F9018950F931F93CF93DF93D8
:10390000EC0104970CF05EC0F894509A589885E04A
:103910008A95F1F700009C2F969595708C2F8570F5
:10392000980F892F837096959695292F93E0CC0F49
:10393000DD1F9A95E1F7280F822F8C2B082FB0DE20
:1039400000C068E0802F03DF80E18A95F1F750988E
:10395000589A489B30C087E090E048992EC0FE01FD
:10396000ED5FFE4F6381611559F02091A701309101
:10397000A80184819581820F931FC2DE8115F9F021
:1039800087DE80E28A95F1F75898509A80E18A950F
:10399000F1F7CD5FDE4F6881611549F02091A701F5
:1039A0003091A80189819A81820F931FF2DE78DE1F
:1039B000789481E008C000C0CCCF019749F4509AB8
:1039C000589A789480E0DF91CF911F910F910895DC
:1039D00000C0C3CF08959B01BA019091C8029430F2
:1039E000D9F48F708093E9009FEF8091E80085FD06
:1039F00006C085ED8A95F1F700009150B1F78091EE
:103A0000E80085FF09C040E050E0C901BCD18091C9
:103A1000E8008E778093E800089543E050E0BC0111
:103A200082E0D9CF46E050E0BC0182E0D4CFCF9312
:103A3000DF93EC01BEDC48E050E0BE0181E0CBDF6B
:103A400088E0FE01ACE8B2E001900D928A95E1F7C2
:103A5000DF91CF9108958091C702811107C01AD3D9
:103A60006AD38091E20084608093E200089510920E
:103A7000C702089581DC81E08DCC6091C40281E0B1
:103A8000611101C080E06ACC9091C80281E094305D
:103A900009F080E06091C4026DCC42E061EC81E00D
:103AA00075D242E261EC82E071D29091C80281E06D
:103AB000943009F080E06091C40244CC8091CA0245
:103AC000893081F148F4823009F496C0833009F4DA
:103AD00057C0813041F008958A3009F480C08B309E
:103AE00009F468C008958091C902813A09F047C07D
:103AF0008091E800877F8093E8008091CD029091CB
:103B0000CE02892B59F060E080E090E070E087D130
:103B10008091E8008B778093E800089568E08CE856
:103B200092E0F4CF8091C902813249F58091CD02B3
:103B30009091CE02029718F58091E800877F8093DC
:103B4000E8008091E80082FF16C02091F300809188
:103B5000F200922F029731F48091F100813011F040
:103B6000863019F48091F10027DC8091E8008B7792
:103B70008093E8003FC28091C8028111E2CF08958E
:103B80008091C902813AD9F78091CD029091CE02FD
:103B9000892BA9F78091E800877F8093E8008091C6
:103BA000E80080FFFCCF05DC8093F1008091E80005
:103BB0008E77DECF8091C902813209F78091CD02E4
:103BC0009091CE02892BD9F68091E800877F80936F
:103BD000E80010D28091CB02DDDB0C94AE06809120
:103BE000C902813261F68091E800877F8093E80006
:103BF00001D28091CC02EECB8091C902813A09F0CA
:103C0000BECF8091E800877F8093E8008091E80034
:103C100080FFFCCFEADBC8CF84B7877F84BF0FB6B5
:103C2000F894A8958091600088618093600010925C
:103C300060000FBE80E890E00FB6F89480936100BA
:103C4000909361000FBEA4CB25D275D2E2EEF0E0D6
:103C50008081846080837894D2C485E291E051CAE7
:103C60008091C802853029F48091C802853011F016
:103C7000AACC08957DDCC4DB8115B1F38091C60226
:103C8000811591F36AD00E94AE068FEF99E628E184
:103C9000815090402040E1F700C00000D1DBE4CF2C
:103CA00008959A014091CF025091D00200C0492F4F
:103CB00050E043305105D1F078F44130510509F41A
:103CC0003DC04230510571F48BE390E04EE253E089
:103CD000F90140835183089541325105E9F04232A0
:103CE000510519F180E090E040E0F2CF482F50E01C
:103CF000813061F04230510561F0EAE2F3E04115B4
:103D0000510581F7849190E0AF01E2CFEAE1F3E061
:103D1000F9CFECEEF2E0F6CF61307105A0F011F7CB
:103D200089E090E049E553E0D3CF6130710580F040
:103D3000C9F68BE790E04BE753E0CACF82E190E011
:103D400049E653E0C5CF89E090E040E453E0C0CFBE
:103D500084E490E046EF53E0BBCF80E189BD82E18F
:103D600089BD09B400FEFDCF8091D8008F7D80937E
:103D7000D8008091E00082608093E0008091E000B4
:103D800081FDFCCF0895AF92BF92CF92DF92EF9268
:103D9000FF921F93CF93DF937C01EB016A0149D11E
:103DA000182F811122C0C114D10439F0F60180818D
:103DB0009181C81BD90BE80EF91EA12CB12C2097BC
:103DC000A1F08091E80085FD20C08091E8008E7709
:103DD0008093E800C114D10499F0F60180819181AB
:103DE0008A0D9B1D8083918315E0812FDF91CF91F8
:103DF0001F91FF90EF90DF90CF90BF90AF9008950C
:103E000018D18115F1F2182FF0CFF70181917F01C0
:103E10008093F10021978FEFA81AB80AD0CFFC0148
:103E20008091CF029091D0028617970720F06115FC
:103E3000710561F0CB0140E0009771F441110CC0B5
:103E40008091E80082FF36C080E008958091E8000C
:103E50008E778093E800EECF2091C8022115B1F152
:103E60002530B1F12091E80023FD2EC02091E8001B
:103E700022FDE6CF2091E80020FFDECF4091F30045
:103E80002091F200342F009719F02830310558F0B6
:103E900041E02830310509F040E02091E8002E771C
:103EA0002093E800C9CF41914093F10001972F5F23
:103EB0003F4FE9CF8091C802811541F0853041F034
:103EC0008091E80083FFBCCF81E0089582E00895EF
:103ED00083E00895FC018091CF029091D002861773
:103EE000970720F06115710561F0CB0140E0009764
:103EF00071F441110CC08091E80082FF37C080E06E
:103F000008958091E8008E778093E800EECF2091AD
:103F1000C8022115B9F12530B9F12091E80023FD3F
:103F20002FC02091E80022FDE6CF2091E80020FF7D
:103F3000DECF4091F3002091F200342F009719F06A
:103F40002830310558F041E02830310509F040E0D3
:103F50002091E8002E772093E800C9CF4491409348
:103F6000F100319601972F5F3F4FE8CF8091C80253
:103F7000811541F0853041F08091E80083FFBBCF8F
:103F800081E0089582E0089583E00895982F9730A6
:103F900028F08F708093E90081E008959093E90004
:103FA000242F762F50E0981731F07091EC0020917B
:103FB000ED005091F00021FD02C09F5FE8CF3091ED
:103FC000EB003E7F3093EB003091ED003D7F30936E
:103FD000ED003091EB0031603093EB007093EC001A
:103FE0002093ED005093F0002091EE0027FDE5CFE7
:103FF00080E008958091C90287FF13C08091E80096
:1040000082FF06C08091E8008B778093E8000895D6
:104010008091C8028111F2CF08958091C802811564
:10402000D9F38091E80080FFF8CF8091E8008E7787
:10403000ECCF2091E4003091E50095E6A9012091B4
:10404000EC00822F817020FF06C08091E80080FF85
:1040500006C080E008952091E80022FD1AC08091FA
:10406000C802811589F0853089F08091EB0085FDCB
:104070000FC02091E4003091E50042175307F9F298
:104080009150E1F684E0089582E0089583E0089578
:1040900081E008955FD066D0E0EEF0E0808181603D
:1040A0008083E8ED80818F77808319BCA7EDB0E035
:1040B0008C918E7F8C9380818F7E80831092C7023B
:1040C0000895CF93DF9346D04DD0C8EDD0E08881DE
:1040D0008F77888388818068888388818F7D8883B3
:1040E00019BC1092C8021092C4021092C60210921B
:1040F000C502E0EEF0E080818B7F80838881816063
:10410000888342E060E080E041DFE1EEF0E0808122
:104110008E7F8083E2EE80818160808380818860F1
:104120008083E0EE80818E7F8083888180618883B8
:10413000DF91CF910895E8EDF0E080818F7E80835C
:10414000E7ED80818160808384E082BF81E080939D
:10415000C702B7CFE8EDF0E080818E7F80831092B8
:10416000E20008951092DA001092E10008951F9283
:104170000F920FB60F9211242F933F934F935F939B
:104180006F937F938F939F93AF93BF93EF93FF931F
:104190008091E10082FF0AC08091E20082FF06C0A8
:1041A0008091E1008B7F8093E10028D28091DA003A
:1041B00080FF18C08091D80080FF14C08091DA0081
:1041C0008E7F8093DA008091D90080FF8FC080E1DC
:1041D00089BD82E189BD09B400FEFDCF81E08093F5
:1041E000C80239DC8091E10080FF18C08091E200B4
:1041F00080FF14C08091E2008E7F8093E200809166
:10420000E20080618093E2008091D8008062809318
:10421000D80019BC85E08093C8022FDC8091E100B2
:1042200084FF28C08091E20084FF24C080E189BD22
:1042300082E189BD09B400FEFDCF8091D8008F7D59
:104240008093D8008091E1008F7E8093E10080917F
:10425000E2008F7E8093E2008091E2008160809393
:10426000E2008091C402811509F445C084E0809386
:10427000C8020ADC8091E10083FF27C08091E20040
:1042800083FF23C08091E100877F8093E10082E07B
:104290008093C8021092C4028091E1008E7F8093C7
:1042A000E1008091E2008E7F8093E2008091E20045
:1042B00080618093E20042E060E080E067DE809110
:1042C000F00088608093F000D5DBFF91EF91BF9103
:1042D000AF919F918F917F916F915F914F913F919E
:1042E0002F910F900FBE0F901F90189519BC109230
:1042F000C802BDDB77CF8091E30087FF02C083E077
:10430000B6CF81E0B4CF1F920F920FB60F92112457
:104310001F932F933F934F935F936F937F938F934D
:104320009F93AF93BF93CF93DF93EF93FF93E9EE08
:10433000F0E080811091EC008F7010FB112717F9CD
:10434000182B1082C0EFD0E08881877F8883789413
:104350001CD0E9EEF0E010828881886088831F70AD
:104360001083FF91EF91DF91CF91BF91AF919F911A
:104370008F917F916F915F914F913F912F911F91FD
:104380000F900FBE0F901F901895AAE2B0E0EAECD4
:10439000F1E280C189EC92E0FC0101962091F100EC
:1043A000208322E0813D9207B9F788DB8091E80005
:1043B00083FF37C08091C9029091CA029A3088F574
:1043C000E92FF0E0E95BFB4D50C1803889F082387D
:1043D00041F58091CD028F70873018F58093E90008
:1043E0008091EB0085FB882780F91092E90006C0D8
:1043F0008091C602880F9091C502892B9091E800A8
:10440000977F9093E8008093F1001092F1008091E3
:10441000E8008E7722C0811115C08091CB028130D7
:1044200001F18091E80083FF0AC08091E800877F56
:104430008093E8008091EB0080628093EB00AA9665
:10444000E3E044C1823069F78091CB02811579F0B5
:104450001092E9008091E800877F8093E800CADD30
:10446000E0CF933009F080E08093C602F1CF8091D5
:10447000CD028F70282F2150263098F68093E900C6
:104480002091EB0020FFE4CF933031F48091EB00DA
:1044900080628093EB00DCCF9091EB009061909371
:1044A000EB0021E001C0220F8A95EAF72093EA0091
:1044B0001092EA008091EB008860EBCF8111B1CFC0
:1044C0008091CB028F77182F8091E3008078812B29
:1044D0008093E3008091E800877F8093E8008ADD85
:1044E0008091E80080FFFCCF8091E300806880939A
:1044F000E30083E0111101C082E08093C80291CFF4
:104500008058823008F08DCF8091CB029091CC0200
:104510008C3D23E0920789F583E08A838AE28983D0
:104520004FB7F894DE01139620E03EE051E2E32F0E
:10453000F0E050935700849120FF03C082958F7064
:104540003F5F8F708A30B8F0895C8D931D922F5F2A
:10455000243169F74FBF8091E800877F8093E8009E
:104560006AE270E0CE0101965ADC8091E8008B7718
:104570008093E80056CF805DE8CF6091CD027091C6
:10458000CE029E012F5F3F4FA9018BDBBC01892B1F
:1045900009F447CF9091E800977F9093E8008981D4
:1045A0009A8198DCE2CF803809F03BCF8091E80017
:1045B000877F8093E8008091C4028093F10027CF29
:1045C00081112FCF9091CB02923008F02ACF8091A9
:1045D000E800877F8093E8009093C4020BDD809110
:1045E000C402811529F084E08093C80256DA19CFFD
:1045F0008091E30087FDF7CF81E0F6CF0895CF9358
:104600008091C802811591F08091E900C091EC0081
:104610008F70C0FBCC27C7F9C82B1092E90080919E
:10462000E80083FDB2DECF70C093E900CF9108951A
:1046300031DD1092C80208958091E30087FB88273E
:1046400080F9089597FB072E16F4009406D077FDA5
:1046500008D048D007FC05D03EF4909581959F4F37
:104660000895709561957F4F0895EE0FFF1F059097
:10467000F491E02D09942F923F924F925F926F92A6
:104680007F928F929F92AF92BF92CF92DF92EF92E2
:10469000FF920F931F93CF93DF93CDB7DEB7CA1B63
:1046A000DB0B0FB6F894DEBF0FBECDBF09942A888E
:1046B000398848885F846E847D848C849B84AA8436
:1046C000B984C884DF80EE80FD800C811B81AA81C3
:1046D000B981CE0FD11D0FB6F894DEBF0FBECDBF8E
:1046E000ED010895AA1BBB1B51E107C0AA1FBB1F08
:1046F000A617B70710F0A61BB70B881F991F5A956E
:10470000A9F780959095BC01CD010895FB01DC01CE
:1047100004C08D910190801921F441505040C8F798
:10472000881B990B0895FB01DC0102C001900D92DA
:1047300041505040D8F70895F999FECF92BD81BD00
:10474000F89A992780B50895A8E1B0E042E050E0DA
:1047500020C0262FF999FECF92BD81BDF89A01970E
:1047600000B4021639F01FBA20BD0FB6F894FA9AB9
:10477000F99A0FBE08950396272FECDFEADF252F65
:10478000E9DF242FE7CF0196272FE4DFE2CFDC011A
:10479000CB01FC01F999FECF06C0F2BDE1BDF89A4C
:1047A000319600B40D9241505040B8F70895F894F6
:1047B000FFCFE304E3041A051A0571058D050B0507
:1047C0000B0591050306100610067E137513811361
:1047D0007213671367137213671367139D136713BD
:1047E000A8136713671367136713671372136713AD
:1047F0006713721367138F1367136713BD13BD130A
:10480000BD13BD13BD13BD13BD13BD13BD136A137B
:1048100067137E1371130E157D151615E014E4143D
:104820001A15E8141E152A15F4147615F8142E1509
:10483000FC1432155715001536155E1506153C1576
:104840004415EC142215F01426150A1540154E15C2
:1048500067157415DA14121584151D162216241600
:1048600029163916391639163916391639163916E0
:1048700039162B162F163216371646164C165016AA
:104880005C1862184D18561868186E187418E521CF
:104890000B2211220B2211225E2280221122D3220E
:0248A000E02214
:1048A20026020100000001000000000000000601D5
:1048B20000000004070000000000002808503C0728
:1048C2001400000100E719171DEA1C121D0D1DE25C
:1048D20000E900EA00B500B600B700CD008301CCC4
:1048E200008A019201940121022302240225022658
:1048F2000227022A02B300B4006F0070009F01CBAE
:10490200019F02A002E200E900EA00B500B600B78A
:1049120000CD008301CC008A01920194012102237F
:104922000224022502260227022A02B300B4006FE3
:104932000070009F01CB019F02A002946697C634CB
:0A49420035F6F73133323644020037
:00000001FF
